:020000040000FA
:0400000001303A2869
:08000800A000030EA100831209
:1000100005191028831601178312B23081002B288E
:1000200083160113831203140B190310A80DA90DD5
:10003000AA0DAB0DAC0DAC16FF302C02031D2B2806
:10004000FA302B02031D2B2831152A08AF0029088E
:10005000AE002808AD008B100B11210E8300A00EFE
:04006000200E090065
:0C007400203084008001840A6030040207
:10008000031C3C281230B00077218316FF23900018
:10009000831283160C308505870183128501870141
:1000A000073099000030831691009F008312C830FA
:1000B00083168100831231309000003083168C004B
:1000C000831210308B00831610309B001C141A080A
:1000D0008312BD00DD2181018E018F010B118B1078
:1000E0000B108C018B178320311986205B21B30BF9
:1000F0008128031085190314B90DF0303902031952
:100100000421EE21732864003210080031110130FF
:10011000B7008B132030370783169B001C141A0876
:100120008312A4001030370783169B001C141A0892
:100130008312A300A6000230A606003037078316FC
:100140009B001C141A088312A200A7000130A70606
:100150008B17321CB12822090339A200A309A40974
:10016000A50924082F02031DFE2823082E02031DC3
:10017000D92822082D02031DFE2801303702031D55
:10018000C4283D143E147F2102303702031DCB28C2
:10019000BD143E148B2103303702031DD2283D15B8
:1001A0003E14972104303702031DD928BD153E1493
:1001B000A32126082E02031DFE2827082D02031D59
:1001C000FE2801303702031DE8283D103E14AF2100
:1001D00002303702031DEF28BD103E14B821033052
:1001E0003702031DF6283D113E14C12104303702A9
:1001F000031DFD28BD113E14CA21FE28B70A053093
:1002000037020318080089280130B600B300B40093
:10021000B500B70085018701B1138320B30B2A29EC
:10022000031085190314B90DF0303902031951294F
:10023000B41F8501B41F8701B40B2A293708B608FB
:100240000319B60003192829FF3085008700B6037B
:100250009630B400311D0D293111321C34292D097D
:100260000339AD00AE09AF092F1C0D298E018F0196
:100270000C1C0D290C102E1E0D298B132030370756
:10028000BB002F08BA00642110303707BB002E08CE
:10029000BA00642100303707BB002D08BA00642182
:1002A0008B1785018701B70AB60105303702031C99
:1002B0000D29DD2108003E1C08003E101030BB0057
:1002C0003D08BA00642108008B133A0883161C15F8
:1002D0009A003B089B0055309D00AA309D009C145D
:1002E00064009C1870291C1183128B170800831658
:1002F00010309B001C141A088312BD0008003D1426
:10030000B122DC00C122C400D122CC000130C800DF
:10031000FF30C0000800BD14B522DD00C522C500B5
:10032000D522CD000130C900FF30C10008003D15C5
:10033000B922DE00C922C600D922CE000130CA008F
:10034000FF30C2000800BD15BD22DF00CD22C7006E
:10035000DD22CF000130CB00FF30C30008005C1A63
:100360008510DC1A05105C1B8512DC1B05120800C9
:100370005D1A8510DD1A05105D1B8512DD1B051247
:1003800008005E1A8510DE1A05105E1B8512DE1B42
:10039000051208005F1A8510DF1A05105F1B851211
:1003A000DF1B05120800380903398500B800080072
:1003B000380930398500B80008003D187F215C1CE1
:1003C0003D10BD188B215D1CBD103D1997215E1C91
:1003D0003D11BD19A3215F1CBD1108000A300F0299
:1003E000031C08008E018F013D1C1E2AC80B1E2A0B
:1003F0004C08C800C00A4408400203181A2A9D226B
:10040000D0005C1E072A501C851050188514DC1E75
:100410000D2AD01C0510D01805145C1F132A501D7E
:10042000851250198516DC1F1E2AD01D0512D01901
:1004300005161E2AC0015C18FF293D10BD1C482A64
:10044000C90B482A4D08C900C10A450841020318D2
:10045000442AA222D0005D1E312A501C851050185B
:100460008514DD1E372AD01C0510D01805145D1F19
:100470003D2A501D851250198516DD1F482AD01DB2
:100480000512D0190516482AC1015D18292ABD1088
:100490003D1D722ACA0B722A4E08CA00C20A4608BB
:1004A000420203186E2AA722D0005E1E5B2A501C4F
:1004B000851050188514DE1E612AD01C0510D01836
:1004C00005145E1F672A501D851250198516DE1F00
:1004D000722AD01D0512D0190516722AC2015E18A3
:1004E000532A3D11BD1D9C2ACB0B9C2A4F08CB00E3
:1004F000C30A470843020318982AAC22D0005F1EA3
:10050000852A501C851050188514DF1E8B2AD01C9C
:100510000510D01805145F1F912A501D851250191F
:100520008516DF1F9C2AD01D0512D01905169C2A9E
:10053000C3015F187D2ABD11080003308A004008FE
:10054000003E820003308A004108403E82000330B2
:100550008A004208803E820003308A004308C03E81
:10056000820003308A003730820003308A007730FF
:10057000820003308A00B730820003308A00F730EF
:10058000820003308A003530820003308A007530E3
:10059000820003308A00B530820003308A00F530D3
:1005A000820003308A003630820003308A007630C1
:1005B000820003308A00B630820003308A00F630B1
:0205C0008200B7
:100600000134023403340434053406340734083426
:1006100009340A340B340C340D340E340F341034D6
:100620001134123413341434153416341734183486
:1006300019341A341B341C341D341E341F34203436
:1006400021342234233424342534263427342834E6
:1006500029342A342B342C342D342E342F34303496
:100660003134323441344234433432342834F13476
:100670008034803480348034803480348034FF345B
:1006800001340234033404340534063407340834A6
:1006900009340A340B340C340D340E340F34103456
:1006A0001134123413341434153416341734183406
:1006B00019341A341B341C341D341E341F342034B6
:1006C0002134223423342434253426342734283466
:1006D00029342A342B342C342D342E342F34303416
:1006E0003134323480348034803432341E34303407
:1006F0008034803480348034803480348034FF34DB
:100700000134023403340434053406340734083425
:1007100009340A340B340C340D340E340F341034D5
:100720001134123413341434153416341734183485
:1007300019341A341B341C341D341E341F34203435
:1007400021342234233424342534263427342834E5
:1007500029342A342B342C342D342E342F34303495
:100760003134323480348034803432340A34F134D9
:100770008034803480348034803480348034FF345A
:1007800001340234033404340534063407340834A5
:1007900009340A340B340C340D340E340F34103455
:1007A0001134123413341434153416341734183405
:1007B00019341A341B341C341D341E341F342034B5
:1007C0002134223423342434253426342734283465
:1007D00029342A342B342C342D342E342F34303415
:1007E0003134323480348034803432341434F1344F
:0E07F00080348034803480348034803480340F
:084000000F000300050003009E
:02400E00CC01E3
:10420000010078007A007C007E007B0079007F004E
:104210007D007A0078007E007C00FF00FF00FF0038
:104220000000F200F600FA00FE00F200F600FA00CC
:10423000FE00F200F600FA00FE00FF00FF00FF00A3
:10424000010005000500050005000900090009003E
:1042500009000D000D000D000D00FF00FF00FF0024
:10426000FF00FF00FF00FF00FF00FF00FF00FF0056
:10427000FF00FF00FF00FF00FF00FF00FF00FF0046
:10428000FF00FF00FF00FF00FF00FF00FF00FF0036
:10429000FF00FF00FF00FF00FF00FF00FF00FF0026
:1042A000FF00FF00FF00FF00FF00FF00FF00FF0016
:1042B000FF00FF00FF00FF00FF00FF00FF00FF0006
:1042C000FF00FF00FF00FF00FF00FF00FF00FF00F6
:1042D000FF00FF00FF00FF00FF00FF00FF00FF00E6
:1042E000FF00FF00FF00FF00FF00FF00FF00FF00D6
:1042F000FF00FF00FF00FF00FF00FF00FF00DD00E8
:00000001FF
